:10000000A4C00000BFC00000BDC00000BBC0000015
:10001000B9C00000B7C00000B5C00000B3C0000008
:10002000B1C00000AFC00000D3C40000ABC00000EE
:10003000A9C00000A7C00000A5C00000A3C0000028
:10004000A1C000009FC000009DC000009BC0000038
:1000500099C0000097C0000095C0000093C0000048
:1000600091C000008FC000008DC000008BC0000058
:1000700089C0000087C0000085C0000083C0000068
:1000800081C000007FC000007DC000007BC0000078
:1000900079C0000077C0000005010906A10105072D
:1000A00019E029E7150025017501950881029501E0
:1000B00075082565190029658100C012010002003C
:1000C0000000400000424B0000010203010902222F
:1000D00000010100C0320904000001030001000911
:1000E00021011000012223000705810308000204FA
:1000F0000309042203440065006E00760065007267
:10010000002000470069006E00670065007200690A
:10011000006300680028034D007900550053004239
:100120000020004B006500790062006F00610072E2
:100130000064002000440065006D006F000C033077
:10014000002E0031002E0030000011241FBECFEF22
:10015000D0E2DEBFCDBF11E0A0E0B1E0E2E4FBE021
:1001600000E00BBF02C007900D92A830B107D9F78D
:1001700015E0A8E0B1E001C01D92A231B107E1F79E
:1001800021D0DEC43DCF9C01809111058823C9F0A8
:10019000809110058823A9F081E08093E900809187
:1001A000E80085FF0EC02093F1003093F1008091AC
:1001B000E8008E7F8093E8008091E8008F7780933D
:1001C000E8000895CFEFD0E2DEBFCDBF80E8809396
:1001D00061001092610087B1867E87B988B189611C
:1001E00088B98AB1806F8AB98BB18F708BB98BB1A6
:1001F0008F7080698BB960E081E07DD182E080936F
:100200000B0510E0E12FFF27EE0FFF1FEE0FFF1F82
:10021000E050FF4F8381882321F00180F281E02D9F
:1002200009951F5F123070F3ECCFCF92DF92EF92FF
:10023000FF920F931F93CF93DF9386B180958971BF
:1002400084FF5AC0409108015091090122C086B133
:1002500080958971992784FF1EC083FDF8CFFA012C
:10026000E65FFE4F80FD02C087E201C08EE1808321
:100270004F5F5F4F84E04030580710F040E050E09F
:1002800086B180958971282F332724FF04C023FF6E
:10029000F7CF84FDDCCF5093090140930801C0E003
:1002A000C0900801D0900901EE24FF2414C0F7018A
:1002B000E65FFE4FD081CE0166DF00E117E2C801A4
:1002C0000197F1F7D0E0CE015EDFC8010197F1F7A9
:1002D0000894E11CF11CEC14FD0449F7D8E2CE01AE
:1002E00052DF80E197E20197F1F7D0E0CE014BDFDA
:1002F0001092090110920801DF91CF911F910F9187
:10030000FF90EF90DF90CF90089540E061EC81E0A6
:1003100020D18BB18F7080668BB90895CF93DF9316
:10032000DA01E9018330E9F0843030F4813059F0AA
:10033000823009F04CC00EC0813209F436C08232DE
:1003400009F045C03DC08BEB90E08D939C9382E11A
:1003500090E031C08DEC90E08D939C9382E290E030
:100360002AC0613071F0613028F0623081F0633072
:1003700071F515C08FEE90E08D939C9384E090E032
:100380001AC0E3EFF0E0ED93FC93E49105C0E5E1E2
:10039000F1E0ED93FC93E4918E2F99270CC0EDE3EF
:1003A000F1E0ED93FC93E491F7CF8FED90E08D9326
:1003B0009C9389E090E09983888381E090E009C074
:1003C00088E990E08D939C9383E290E0F4CF80E005
:1003D00090E0DF91CF910895809111058111AFD305
:1003E0001092A0001092E2001092DE008091D800DE
:1003F0008E7F8093D800CCD08091E0008160809384
:10040000E000109211051092100510920F0508954A
:10041000E3DF1092A0001092E2001092DE00B8D04C
:1004200080910A05813091F480910E0580FF04C00F
:100430008091E000846003C08091E0008B7F809316
:10044000E0008091D80081608093D8008091D7002F
:1004500081608093D7008EE089BD09B400FEFDCF96
:100460008091D8008F778093D8008091D8008068E1
:100470008093D8008091D8008F7D8093D80040E38E
:1004800060E080E066D08823B9F08091E0008E7F44
:100490008093E0008091E20081608093E20080918F
:1004A000E20088608093E20081E080931005109262
:1004B000110581E090E0089581E041D380E090E073
:1004C00008958ADF10920A0510920E05E8EDF0E01B
:1004D00080818F77808319BCA7EDB0E08C918E7FEF
:1004E0008C9380818F7E808380818D7F80838081CB
:1004F0008E7F808308950F931F93182F062F80916E
:1005000010058111DEDF10930A05112319F480E034
:1005100016D31CC0113019F081E011D305C08091B1
:10052000D70080688093D70081E0809310051092F7
:1005300011058091D80080618093D80000930E054A
:100540008091D80081608093D80078941F910F919A
:10055000089587708093E9008091EB00816080931B
:10056000EB006093EC008091ED008270842B80930F
:10057000ED008091ED0082608093ED008091EE00AF
:10058000992787FD90958827990F881F99270895A7
:1005900020E030E0822F87708093E9008091ED00A9
:1005A0008D7F8093ED008091EB008E7F8093EB0038
:1005B0002F5F3F4F2730310569F708959091F10083
:1005C0008091E3009F738078982B9093E300809153
:1005D000E800877F8093E8008091E8008E7F809319
:1005E000E8008091E8008F778093E8008091E80030
:1005F00080FFFCCF8091E30080688093E300089542
:100600008091E800877F8093E80080910F058093B8
:10061000F1008091E8008E7F8093E8008091E800EF
:100620008F778093E8008091E80082FFFCCF809173
:10063000E8008B7F8093E8008091E8008F778093BB
:10064000E8000895CF93DF93CDB7DEB721970FB6BB
:10065000F894DEBF0FBECDBF9091F10099839091C9
:10066000F10099832091F10099278F71907081306A
:10067000910539F08230910531F0892B99F593E09D
:100680000BC090E009C027702093E9009091EB0027
:10069000909591701092E9008091E800877F809397
:1006A000E8009093F1001092F1008091E8008E7FB5
:1006B0008093E8008091E8008F778093E800809134
:1006C000E80082FFFCCF8091E8008B7F8093E800F8
:1006D0008091E8008F778093E8008091E800877F21
:1006E0008093E80021960FB6F894DEBF0FBECDBF11
:1006F000DF91CF910895CF93DF93CDB7DEB72197E8
:100700000FB6F894DEBF0FBECDBF2091F1009091DF
:10071000F10099839091F1008F718230B9F4222316
:10072000A9F4892F877091F08093E9008091EB0004
:1007300080FD0AC08091EB0081608093EB00809186
:10074000E800877F8093E8001092E90021960FB6B9
:10075000F894DEBF0FBECDBFDF91CF910895CF9348
:10076000DF93CDB7DEB721970FB6F894DEBF0FBE8B
:10077000CDBF2091F1009091F10099839091F1000B
:100780008F718230B9F42223A9F4892F877091F0F8
:100790008093E9008091EB0080FF0AC08091EB001C
:1007A0008E7F8093EB008091E800877F8093E80044
:1007B0001092E90021960FB6F894DEBF0FBECDBFB0
:1007C000DF91CF910895CF93DF93CDB7DEB7259713
:1007D0000FB6F894DEBF0FBECDBF6091F1008091DF
:1007E000F1009E012C5F3F4FAE014E5F5F4F96DDE3
:1007F000882309F472C08091F10089838091F1000F
:1008000089832091F1008091F1009927582F442786
:100810003327422B532B8091E800877F8093E80099
:100820002C813D812417350760F42F733070232B02
:1008300011F4A1E001C0A0E06A817B812C813D819F
:1008400023C05D834C83F7CF8091E80080FFFCCF0D
:10085000FB0190E006C09F5F84918093F100319688
:100860009A01BF012115310529F0A90141505040DD
:10087000903489F78091E8008E7F8093E800809122
:10088000E8008F778093E8002115310521F08091F1
:10089000E80082FFD9CF8091E80082FD14C0AA232E
:1008A00071F08091E80080FFFCCF8091E8008E7F9E
:1008B0008093E8008091E8008F778093E800809132
:1008C000E80082FFFCCF8091E8008B7F8093E800F6
:1008D0008091E8008F778093E80025960FB6F89412
:1008E000DEBF0FBECDBFDF91CF9108958091F100A3
:1008F000823090F480930F058091E800877F809389
:10090000E8008091E8008E7F8093E8008091E80005
:100910008F778093E800F9CC08956091F100262F3D
:1009200033278091F100853081F0863038F48130B2
:1009300051F18130C0F0833071F51DC0883069F00D
:10094000893039F0863039F50CC0662321F536DE62
:1009500023C0662301F5CADF1FC06038E1F450DE12
:100960001BC031DF19C02F7930702338310599F45D
:10097000862F68DE11C02F7930702330310559F48D
:10098000862FB9DE09C02F7930702330310519F474
:10099000862FE5DE01C0D3D08091E80083FF0AC036
:1009A0008091EB0080628093EB008091E800877F6C
:1009B0008093E800089580911105882331F010920A
:1009C000E9008091E80083FDA8CF0895F4CF089551
:1009D0001F920F920FB60F9211242F933F934F93B4
:1009E0005F936F937F938F939F93AF93BF93EF9397
:1009F000FF938091DA0080FF2EC08091D80080FFA5
:100A00002AC08091DA008E7F8093DA0098D080919E
:100A1000D90080FD94D080911105882381F48091C4
:100A2000D90080FF0CC080911005882341F0F0DCD4
:100A3000882389F081E08093110581D00CC08091DA
:100A40000A05813029F48091E00081608093E00004
:100A500076D0109211058091E10080FF1AC080913C
:100A6000E20080FF16C08091E1008E7F8093E1005C
:100A70008091D80080628093D80019BC8091E200F8
:100A80008E7F8093E2008091E20080618093E2009B
:100A900056D08091E10084FF1EC08091E20084FF67
:100AA0001AC08091E1008F7E8093E1008091D80090
:100AB0008F7D8093D8008EE089BD09B400FEFDCF04
:100AC0008091E2008F7E8093E2008091E20081605D
:100AD0008093E20034D08091E10083FF1FC08091B9
:100AE000E20083FF1BC08091E100877F8093E100DB
:100AF00010920F058091E1008E7F8093E10080913C
:100B0000E2008E7F8093E2008091E200806180931A
:100B1000E20040E360E080E01CDD11D0FF91EF9146
:100B2000BF91AF919F918F917F916F915F914F9105
:100B30003F912F910F900FBE0F901F901895089521
:020B4000FFCFE5
:080B420000E6040101150101A8
:00000001FF
